:020000040000FA
:02000000040AF0
:080008003B0C06008F0C020006
:1000100046046800690066060B0A0602030E2D00FE
:1000200003046D030D023109E9010306A8028D02E4
:100030003109E801030408032C0003040C033A0906
:100040002F0003042F0303042F03AF02410C2E00E3
:100050000F02AE00EE022A0A4605EF022D0A460400
:100060000B0AE201AB0805089E080708C10808084A
:1000700032080608E20180088C089808A508B00834
:10008000BC08C608D008DA08E208EA08F008F50853
:10009000FA08FD08FE08FF08FE08FD08FA08F50842
:1000A000F008EA08E208DA08D008C608BC08B00878
:1000B000A50898088C088008730867085A084F0834
:1000C000430839082F0825081D0815080F080A08D5
:1000D00005080208010800080108020805080A08C6
:1000E0000F0815081D0825082F08390843084F0870
:0600F0005A0867087308BE
:021FFE00E90FE9
:00000001FF
